:020000040000FA
:04000000E7EF02F034
:0400080013EF13F0EF
:0800180068EF13F00F0B756F88
:10002000000EF76E360EF66E7551F626D8B0F72A2A
:100030000800F55012003031323334353637383954
:10004000414243444546000EF86E270EF76EE00E1F
:10005000F66EAAEC0DF0B9EC16F076EC00F003E3C6
:100060004C6A4D6A04D00AC24CF00BC24DF03CEC15
:1000700019F0B3EC1AF09BEC1DF033EC21F0040EF8
:100080006B6F020E6C6FD5EC20F026EF20F0000EA7
:10009000F86E270EF76ED00EF66EAAEC0DF07DC04E
:1000A000AAF17EC0ABF17FC0ACF180C0ADF181C0E0
:1000B000AEF18DEC22F002EC23F076EC00F013E3CD
:1000C0004C6A4D6A4E6A4F6A506A4CC0AFF14DC0DF
:1000D000B0F14EC0B1F14FC0B2F150C0B3F1030E58
:1000E0004C6E4CC0B9F1D2EC24F0120081C04CF03F
:1000F000D8804CAED890120089EC00F0D5EC01F01D
:100100009EEC01F077EC01F023EC00F047EC00F0FE
:100110001200000EF86E270EF76EAE0EF66EAAEC09
:100120000DF0B9EC16F01CC04CF01DC04DF01BECEE
:1001300021F0030E6B6F26EC20F0000EF86E270EF8
:10014000F76EB20EF66EAAEC0DF0B9EC16F01BC00D
:100150004CF01BEC21F0030E6B6F26EC20F01A66BE
:1001600010D0000EF86E270EF76EEE0EF66EAAECAB
:100170000DF0000EF86E270EF76EF40EF66EAAEC78
:100180000DF0010E1A6210D0000EF86E270EF76EF9
:10019000FA0EF66EAAEC0DF0000EF86E280EF76E51
:1001A000000EF66EAAEC0DF0020E1A6210D0000ED0
:1001B000F86E280EF76E060EF66EAAEC0DF0000E25
:1001C000F86E280EF76E0C0EF66EAAEC0DF0030E0C
:1001D0001A6210D0000EF86E280EF76E120EF66E30
:1001E000AAEC0DF0000EF86E280EF76E180EF66EE3
:1001F000AAEC0DF0040E1A6210D0000EF86E280E54
:10020000F76E1E0EF66EAAEC0DF0000EF86E280EBC
:10021000F76E240EF66EAAEC0DF0050E1A6210D0E1
:10022000000EF86E280EF76E2A0EF66EAAEC0DF090
:10023000000EF86E280EF76E300EF66EAAEC0DF07A
:100240001200000EF86E270EF76EBE0EF66EAAECC8
:100250000DF0A5C161F0A6C162F0A7C163F0A8C10D
:1002600064F0A9C165F033EC21F0050E6B6F010E4F
:100270006C6FD5EC20F026EC20F0040E09EC0DF0AC
:10028000000EF86E270EF76ECA0EF66EAAEC0DF091
:100290009BC161F09CC162F09DC163F09EC164F09E
:1002A0009FC165F033EC21F0050E6B6F010E6C6F92
:1002B000D5EC20F026EC20F098EC0DF0A0C161F018
:1002C000A1C162F0A2C163F0A3C164F0A4C165F052
:1002D00033EC21F0050E6B6F010E6C6F6E85D5EC63
:1002E00020F026EC20F06A0E09EC0DF01200540EFE
:1002F00096EC0DF0460E09EC0DF03150300909EC8A
:100300000DF03A0E09EC0DF0B9EC16F0C5C14CF049
:10031000C6C14DF00A0E516EBBEC1EF01BEC21F075
:10032000050E6B6F6F8726EC20F0000EF86E280E1E
:10033000F76E3A0EF66EAEEC0DF01200356608D090
:10034000000EF86E270EF76E860EF66EAAEC0DF014
:10035000010E356208D0000EF86E270EF76E8E0E75
:10036000F66EAAEC0DF0030E356208D0000EF86EA2
:10037000270EF76E960EF66EAAEC0DF0040E35629F
:1003800008D0000EF86E270EF76E9E0EF66EAAECE1
:100390000DF0020E356208D0000EF86E270EF76ED3
:1003A000A60EF66EAAEC0DF01200000EF86E270EE7
:1003B000F76EDC0EF66EAAEC0DF0B9EC16F02FC05D
:1003C0004CF01BEC21F0010E6B6F26EF20F0716FEB
:1003D000670E96EC0DF0715109EF0DF0235202E11A
:1003E000078C2FD081A0FAD7060E716F20EC0CF08D
:1003F00081A026D0712FFAD71EEC0CF04C6A080EA3
:10040000716F81A009D0D8804C32235202E1078C51
:1004100018D081B0FAD708D0D8904C32235202E1DC
:10042000078C0FD081A0FAD71CEC0CF0712FE9D704
:10043000235202E1078C05D081B0FAD7D89001D0C1
:10044000D8801200079C12EE0CF0130E726F736BC3
:1004500073C0E6FF722FFCD73E0EE7EC01F012EE00
:100460000CF0130E726F736B320E236EB7DF07BC86
:1004700047D04CC0E6FF722FF7D7120E716F12EE05
:100480000CF0516AE6CF4CF04C50511A712FFAD74C
:1004900051C073F0E7CFE8FF515C0AE0000EF86E40
:1004A000270EF76EE60EF66EAAEC0DF0078C28D03C
:1004B00012EE0CF0E6CF4CF0AA0E4C5CFBE0E552DD
:1004C000E6CF2FF0E6CF1AF0E6CF1BF0E6CF1CF018
:1004D000E6CF1DF0E6CF0AF2E6CF0BF2E6CF7DF0D5
:1004E000E6CF7EF0E6CF7FF0E6CF80F0E6CF81F07A
:1004F000E6CFC5F1E6CFC6F1E6CF31F0E6CFC9F1E0
:10050000200EE7EC01F007821200350E0C6EA3EC12
:1005100009F014EC0CF0380E0C6EA3EC09F014EC9E
:100520000CF00C0E0C6EA3EC09F018EC0CF022ECA5
:1005300002F00880140E2A6E12001F0E96EC0DF0C9
:100540005B0E09EC0DF010EE10F0060E716FE6CFA9
:100550004CF00A0E4C6203D02A0E4C6E14D00B0ED7
:100560004C6203D0300E4C6E0ED00C0E4C6203D099
:10057000230E4C6E08D0000E4C6203D0200E4C6E41
:1005800002D0300E4C124C5009EC0DF0712FDFD719
:100590005D0E09EC0DF01200106A116A126A136AFE
:1005A000146A156A10EE10F0E1CF0EF0E2CF0FF0F2
:1005B0001200D2EC02F00788320E226E520EE7ECE7
:1005C00001F0078A0880140E2A6E2D6812002EECA6
:1005D0000CF0C1EC0EF090EC0CF083EC0EF07CEC27
:1005E00000F0CCEC02F09DEC02F0520EE7EC01F0D2
:1005F0000C0E0C6EA3EC09F006EC0CF0050E2E6E42
:1006000085EC02F007AC2ED08EEC0DF0000EF86EEB
:10061000290EF76EA20EF66EAAEC0DF0000EF86E23
:10062000290EF76EB80EF66EAAEC0DF0000EF86EFD
:10063000290EF76ECE0EF66EAAEC0DF0000EF86ED7
:10064000290EF76EE40EF66EAAEC0DF02E5030096E
:1006500009EC0DF002EC0CF08EEC0DF07CEC00F0EF
:100660002E2ECED77CEC00F02E8CB5EC0DF0D8A061
:100670008CD3C8EC0DF00F0E0C6498D08EEC0DF0FE
:10068000190E0C6221D0000EF86E280EF76E500E77
:10069000F66EAAEC0DF0000EF86E280EF76E600EE6
:1006A000F66EAAEC0DF0000EF86E280EF76E760EC0
:1006B000F66EAAEC0DF0000EF86E280EF76E8C0E9A
:1006C000F66EAAEC0DF056D0180E0C6221D0000E7A
:1006D000F86E280EF76EA20EF66EAAEC0DF0000E64
:1006E000F86E280EF76EB40EF66EAAEC0DF0000E42
:1006F000F86E280EF76ECA0EF66EAAEC0DF0000E1C
:10070000F86E280EF76EE00EF66EAAEC0DF032D001
:10071000170E0C6221D0000EF86E280EF76EF60E42
:10072000F66EAAEC0DF0000EF86E290EF76E080EAC
:10073000F66EAAEC0DF0000EF86E290EF76E1E0E86
:10074000F66EAAEC0DF0000EF86E290EF76E340E60
:10075000F66EAAEC0DF00ED0000EF86E280EF76EB5
:10076000460EF66EAAEC0DF00CC0E8FF0F0B300938
:1007700009EC0DF00CC00DF02DEC0EF008EC0CF0B7
:1007800028EC0EF0C8EC0DF00CC0E8FF0F0B3009A0
:1007900009EC0DF00D38F00B0D6E0C500F0B0D1217
:1007A000CEEC0EF08EEC0DF00C6AEFD20EC0E1FF35
:1007B0000FC0E2FF0CC0E6FFE1CF0EF0E2CF0FF07A
:1007C0001A0E0E5CD8B4D2EC02F00C0E0C6203D000
:1007D000D9EC02F002D09EEC09F0A3EC09F00C0E6B
:1007E000106203D0D9EC02F0226A050E106228D004
:1007F000090E116225D00C0E126222D0226A0798CF
:100800008EEC0DF0000EF86E2A0EF76E1E0EF66ED0
:10081000AAEC0DF0000EF86E2A0EF76E340EF66E8E
:10082000AAEC0DF0000EF86E290EF76EF40EF66EBF
:10083000AAEC0DF028EC0EF08EEC0DF0CCEC02F0F2
:10084000070E106205D0CCEC02F01B661B0638D0F8
:100850000A0E106206D0CCEC02F01B2A01E11B68E4
:100860002FD0080E106208D0CCEC02F01A2A060E27
:100870001A5C01E11A6A24D0060E10620ED0CCEC8C
:1008800002F01C6603D01D6601D006D01C061C2891
:10089000D8B41D06D8B41C5213D0090E106212D061
:1008A000CCEC02F0830E4C6E030E4D6E1D504D5C71
:1008B00002E11C504C5CD8B403D01C2AD8B41D2AC9
:1008C00089EC00F0040E106226D0090E116223D0CC
:1008D0000C0E126220D08EEC0DF0000EF86E2A0E77
:1008E000F76E4A0EF66EAAEC0DF0000EF86E2A0EA8
:1008F000F76E600EF66EAAEC0DF0000EF86E2B0E81
:10090000F76EC00EF66EAAEC0DF097EC09F08EECC7
:100910000DF0D9EC02F0040E10622AD0050E11621F
:1009200027D00C0E126201D003D00C0E136220D01F
:100930008EEC0DF0000EF86E2A0EF76E4A0EF66E73
:10094000AAEC0DF0000EF86E2A0EF76E760EF66E1B
:10095000AAEC0DF0000EF86E2B0EF76EC00EF66EC0
:10096000AAEC0DF097EC09F08EEC0DF0D9EC02F04A
:10097000040E106289D0060E116286D08EEC0DF046
:10098000000EF86E2A0EF76E4A0EF66EAAEC0DF007
:10099000000EF86E2A0EF76E8C0EF66EAAEC0DF0B5
:1009A0000C0E126209D0000EF86E2A0EF76EA20E1F
:1009B000F66EAAEC0DF02BD00C0E136265D00B0E68
:1009C000126211D0000EF86E2A0EF76E8C0EF66EC3
:1009D000AAEC0DF0000EF86E2A0EF76EE60EF66E1B
:1009E000AAEC0DF014D0000EF86E2A0EF76ECE0EA3
:1009F000F66EAAEC0DF01250300909EC0DF0000E65
:100A0000F86E2A0EF76EDE0EF66EAAEC0DF0000EF2
:100A1000F86E2B0EF76E120EF66EAAEC0DF008ECC7
:100A20000CF08A8285EC09F00BE2000EF86E2B0EBA
:100A3000F76E280EF66EAAEC0DF08CEC09F002E3CE
:100A40002DEC0EF08A928EEC0DF0000EF86E2A0E50
:100A5000F76E4A0EF66EAAEC0DF0000EF86E2A0E36
:100A6000F76E8C0EF66EAAEC0DF0000EF86E2A0EE4
:100A7000F76EFC0EF66EAAEC0DF006EC0CF08EECA8
:100A80000DF00884D9EC02F0040E10625CD0070E61
:100A9000116259D08EEC0DF0000EF86E2A0EF76E32
:100AA0004A0EF66EAAEC0DF0000EF86E2A0EF76EE6
:100AB000B80EF66EAAEC0DF00C0E126244D0000EC9
:100AC000F86E2A0EF76EA20EF66EAAEC0DF0000E6E
:100AD000F86E2B0EF76E120EF66EAAEC0DF008EC07
:100AE0000CF08A8285EC09F00BE2000EF86E2B0EFA
:100AF000F76E280EF66EAAEC0DF08CEC09F002E30E
:100B00002DEC0EF08A928EEC0DF0000EF86E2A0E8F
:100B1000F76E4A0EF66EAAEC0DF0000EF86E2A0E75
:100B2000F76EB80EF66EAAEC0DF0000EF86E2A0EF7
:100B3000F76EFC0EF66EAAEC0DF006EC0CF08EECE7
:100B40000DF0D9EC02F0050E106232D0010E1162E8
:100B50002FD00C0E13622CD08EEC0DF0000EF86E20
:100B60002A0EF76E4A0EF66EAAEC0DF0000EF86E25
:100B70002B0EF76E3E0EF66EAAEC0DF0000EF86E20
:100B80002B0EF76ED60EF66EAAEC0DF0000EF86E78
:100B90002B0EF76EEC0EF66EAAEC0DF0125030092B
:100BA00009EC0DF097EC09F08EEC0DF0D9EC02F0A9
:100BB000050E106239D0020E116236D00C0E14628E
:100BC00033D08EEC0DF0000EF86E2A0EF76E4A0E42
:100BD000F66EAAEC0DF0000EF86E2B0EF76EF20E0C
:100BE000F66EAAEC0DF0000EF86E2B0EF76ED60E18
:100BF000F66EAAEC0DF0140E96EC0DF012503009C2
:100C000009EC0DF0000EF86E2B0EF76EEC0EF66E82
:100C1000AAEC0DF01350300909EC0DF097EC09F037
:100C20008EEC0DF0D9EC02F0050E106229D0040E06
:100C3000116226D0070E126223D00C0E136220D050
:100C40008EEC0DF0000EF86E2A0EF76E4A0EF66E60
:100C5000AAEC0DF0000EF86E2B0EF76E6A0EF66E13
:100C6000AAEC0DF0000EF86E2B0EF76EC00EF66EAD
:100C7000AAEC0DF097EC09F08EEC0DF0D9EC02F037
:100C8000050E106229D0040E116226D0090E1262E0
:100C900023D00C0E136220D08EEC0DF0000EF86EF7
:100CA0002A0EF76E4A0EF66EAAEC0DF0000EF86EE4
:100CB0002B0EF76E540EF66EAAEC0DF0000EF86EC9
:100CC0002B0EF76EC00EF66EAAEC0DF097EC09F045
:100CD0008EEC0DF0D9EC02F0050E106226D0040E59
:100CE000116223D00C0E126220D08EEC0DF0000E9B
:100CF000F86E2A0EF76E4A0EF66EAAEC0DF0000E94
:100D0000F86E2B0EF76E800EF66EAAEC0DF0000E4C
:100D1000F86E2B0EF76EC00EF66EAAEC0DF097EC87
:100D200009F08EEC0DF0D9EC02F0050E106215D032
:100D3000040E116212D00B0E12620FD00C0E136251
:100D40000CD08EEC0DF0CCEC02F0079A226ABCECD1
:100D500008F08EEC0DF0D9EC02F0050E106212D006
:100D6000050E11620FD00C0E12620CD08EEC0DF03D
:100D7000CCEC02F0079A226A05EC09F08EEC0DF03B
:100D8000D9EC02F09DEC02F00C6A07BE06D094ECA0
:100D90000EF0D8A002D01AEC0AF02E4E2E8C010EC6
:100DA0002E6207D007A205D07CEC00F09DEC02F08B
:100DB0000792020E2E6214D007AE12D0AEEC0AF0EB
:100DC000079E346A010E35620BD0610E96EC0DF071
:100DD0002A0E07A6200E09EC0DF00776C80E256E28
:100DE000030E2E6208D0030E356205D0296603D0AB
:100DF000296878EC0EF0040E2E6207D008A005D00A
:100E00002A6603D008906BEC08F0050E2E6200D025
:100E1000060E2E6200D0070E2E6203D0256601D08A
:100E20000896080E2E620BD0010E356208D0266699
:100E300006D008A604D0ABEC0EF0640E266E090EA8
:100E40002E6211D0010E35620ED026660CD008B687
:100E50000AD0B6EC0EF012EC0CF0ABEC0EF0640E17
:100E6000266EC80E256E0A0E2E6207D0246605D0A7
:100E700007A003D0BAEC09F007900B0E2E622FD01A
:100E800031A02DD007B02BD0C5C14CF0C6C14DF05C
:100E9000C7C151F0C8C152F0B80E536E0B0E546E5C
:100EA0005250545C02E15150535CD8A018D0AA0EA5
:100EB000536E000E546E5250545C02E15150535C1C
:100EC000D8B00DD052504D5C02E151504C5CD8B4BA
:100ED00006D0520EE7EC01F0640E246E07800C0E73
:100EE0002E620DD007AC0BD0079C320E236E23521E
:100EF00003E0B5EC0DF0FBE38EEC0DF007820D0E78
:100F00002E6200D00E0E2E621BD0226619D007A8CA
:100F10000DD0106A116A126A136A146A156A166A89
:100F2000176A186A196A9DEC02F0079807AA08D098
:100F3000079A85EC02F008A403D0A2EC07F008940D
:100F400035EF03F0B9EC16F01CC04CF01DC04DF0AD
:100F5000640E516E2FEC1FF04CC074F0B9EC16F01B
:100F60001CC04CF01DC04DF0716B746702D07183D2
:100F70004DD0010E746305D0640E516E7181718382
:100F800043D0020E746305D0C80E516E7181718317
:100F90003BD0030E746307D02C0E516E010E526EBF
:100FA0007181718331D0040E746307D0900E516E3D
:100FB000010E526E7181718327D0050E746307D0C4
:100FC000F40E516E010E526E718171831DD0060EAA
:100FD000746307D0580E516E020E526E7181718388
:100FE00013D0070E746307D0BC0E516E020E526E02
:100FF0007181718309D0080E746306D0200E516E82
:10100000030E526E718100D037EC1AF071A106D038
:101010000A0E4C6003D016EC08F007D071A305D07F
:101020005A0E4C6402D037EC08F012008EEC0DF032
:1010300058EC08F0000EF86E2C0EF76E340EF66EBB
:10104000AAEC0DF0000EF86E2C0EF76E520EF66E36
:10105000AAEC0DF0000EF86E2C0EF76E7E0EF66EFA
:10106000AAEC0DF002EC0CF08EEC0DF012008EEC00
:101070000DF058EC08F0000EF86E2C0EF76E340EE2
:10108000F66EAAEC0DF0000EF86E2C0EF76E680EE0
:10109000F66EAAEC0DF0000EF86E2C0EF76E7E0EBA
:1010A000F66EAAEC0DF002EC0CF08EEC0DF01200D6
:1010B000000EF86E2C0EF76E4A0EF66EAAEC0DF0CE
:1010C000C7EC16F01CC04CF01DC04DF01BEC21F01D
:1010D000FAEC1FF0120019D83BC037F0790E366ECB
:1010E0009CEC08F03AC037F07A0E366E9CEC08F0B3
:1010F00039C037F07B0E366E9CEC08F038C037F004
:101100007C0E366E9CEC08F01200B9EC16F0C5C1EE
:101110004CF0C6C14DF0E80E516E030E526EBBECA2
:101120001EF01BEC21F042C038F043C039F044C03F
:101130003AF045C03BF012007E0EA7EC08F036C036
:10114000E8FFA7EC08F037C0E8FFA7EF08F04C6E07
:101150008A940DD8080E716F4C32D8A08A94D8B0FA
:101160008A8405D8712FF8D78A8401D812009E0E80
:10117000096E092EFED71200000EF86E2A0EF76EC9
:101180004A0EF66EAAEC0DF0000EF86E2B0EF76EFE
:10119000960EF66EAAEC0DF0000EF86E2B0EF76EA2
:1011A000AC0EF66EAAEC0DF0C9C14CF034EC19F09F
:1011B000B3EC1AF033EC21F0030E6B6F6C6B26EC82
:1011C00020F0000EF86E2B0EF76EB60EF66EAAEC3F
:1011D0000DF0D30E4C6E34EC19F0B3EC1AF033EC86
:1011E00021F0030E6B6F6C6B26EC20F0C80E276E9F
:1011F000000E286E286603D0276601D005D0B5EC16
:101200000DF0F8E3C8EC0DF0120089EC00F02DECC5
:1012100012F0F8EC12F022EC09F047EC09F01BECAC
:1012200010F021EC01F0DC0E276E050E286E28660A
:1012300003D0276601D005D0B5EC0DF0F8E3C8EC7B
:101240000DF01200000EF86E270EF76EB60EF66E59
:10125000AAEC0DF005C261F006C262F007C263F0AD
:1012600008C264F009C265F033EC21F0050E6B6F23
:10127000010E6C6FD5EC20F026EC20F0000EF86E1D
:10128000280EF76E420EF66EAEEC0DF01200000E58
:10129000F86E270EF76EBA0EF66EAAEC0DF000C2CD
:1012A00061F001C262F002C263F003C264F004C2E2
:1012B00065F033EC21F0050E6B6F030E6C6FD5EC0F
:1012C00020F026EC20F0000EF86E280EF76E3E0E91
:1012D000F66EAEEC0DF01200000EF86E2C0EF76EEE
:1012E000080EF66EAAEC0DF0000EF86E2C0EF76EDE
:1012F0001E0EF66EAAEC0DF0C8EC0DF0090E0C6295
:1013000002D0D89001D0D8801200B5EC0DF003E2E5
:1013100081A0FBD7D890120081A002D0640E2C6E61
:10132000B5EC0DF003E22C66F7D7D890120012EC62
:101330000CF081B0FCD706EC0CF012000101C76B79
:10134000C86B000112000C38F00B306E8B8A8B8852
:10135000A00E306203D0B00E306E05D0B00E3062F9
:1013600002D0A00E306E30C08CFF8B9A12EC0CF0C5
:101370008B8A120005EC0AF03C0EE7EC01F09DECC4
:1013800002F0200E96EC0DF0B9EC16F0C7C14CF04F
:10139000C8C14DF00A0E516EBBEC1EF01BEC21F0E3
:1013A00000EE44F011EE31F0030E406EEDCF3EF052
:1013B0003E383F6E93EC20F03EC03FF093EC20F0BF
:1013C000402EF4D711EE32F0050E716FE7CFE8FF33
:1013D00009EC0DF0E6CF0CF0B6DF14EC0CF0712F39
:1013E000F5D7230E09EC0DF00C0E0C6EA3EC09F0F2
:1013F0007CEC00F0CCEC02F09DEC02F00CEC0CF07C
:1014000005EC0AF085EC02F012002A0EE7EC01F080
:1014100018EC0CF081A003D0500E2B6EF9D72B6680
:10142000FED7120023EE00F034C0D9FF32C0DFFF38
:10143000342A1200040E35620CD012EC0AF03B0E76
:10144000326202D0078E04D0FA0E346401D0078EC7
:101450001200020E35620CD012EC0AF0FD0E326260
:1014600002D0078E04D0FA0E346401D0078E120029
:10147000030E35620CD012EC0AF03B0E326202D041
:10148000078E04D0FA0E346401D0078E1200010ECC
:10149000356224D0346603D032C000F318D0010E78
:1014A000346203D032C001F312D0020E346203D092
:1014B00032C002F30CD0030E346203D032C003F307
:1014C00006D0040E346203D032C004F300D0342AB4
:1014D000050E346202D0078E08862FD0000E3562CA
:1014E0002CD07E0E325C02E1346A27D0346604D000
:1014F00032C033F0342A21D0790E335C05E11ED896
:101500001CE232C01EF019D07A0E335C05E116D809
:1015100014E232C01FF011D07B0E335C05E10ED80F
:101520000CE232C020F009D07C0E335C06E106D814
:1015300004E232C021F0078E00D0120032500F0BAF
:101540004C6E0A0E4C5C08E23250F00B4C6EA00E52
:101550004C5C02E2D8901200D8801200000E356276
:101560001FD01E52D8A4B9EF0AF01F52D8B4DBEF37
:101570000BF0C7EC16F020C04CF01FC04DF01EC0A1
:101580004EF019EC1AF0C1EC17F0CEEC16F00A0E82
:10159000516E2FEC1FF042C0C7F143C0C8F10BD110
:1015A000010E356221D0B9EC16F003C34CF002C332
:1015B0004DF001C34EF000C34FF019EC1AF0C1EC2E
:1015C00017F0CEEC16F00A0E516EBBEC1EF0CEEC0E
:1015D00016F0100E516E270E526E2FEC1FF042C007
:1015E000C7F143C0C8F1E7D0030E356241D000C354
:1015F0004CF0460E4C62DFD001C34CF0410E4C6201
:1016000001D003D0420E4C6220D0B9EC16F008C3D2
:1016100042F007C343F006C344F005C345F0E8ECCD
:1016200021F019EC1AF001C34CF0410E4C6205D0C8
:1016300042C078F043C079F019D0420E4C6205D018
:1016400042C07AF043C07BF011D0540E4C620ED0F1
:1016500002C37CF0310E7C6305D07AC0C7F17BC039
:10166000C8F104D078C0C7F179C0C8F12968A3D007
:10167000020E35623BD000C34CF0FE0E4C629BD094
:1016800001C34CF0FE0E4C6296D002C34CF0000E2B
:101690004C6291D003C34CF0940E4C628CD004C3C6
:1016A0004CF0000E4C6287D00AC34CF0FD0E4C6229
:1016B00082D0B9EC16F005C34CF006C34DF007C359
:1016C0004EF008C34FF009C350F019EC1AF0C1EC0A
:1016D00017F0CEEC16F0100E516E270E526E2FEC56
:1016E0001FF042C0C7F143C0C8F165D0040E356297
:1016F00062D000C34CF0460E4C622ED001C34CF0B9
:10170000410E4C6201D003D0420E4C6251D00DC349
:101710004CF03B0E4C624CD0B9EC16F008C342F0D2
:1017200007C343F006C344F005C345F0E8EC21F0DD
:1017300019EC1AF001C34CF0410E4C6205D042C0C6
:1017400078F043C079F021D0420E4C627ED742C07F
:101750007AF043C07BF019D05A0E4C6229D001C3F5
:101760004CF05A0E4C6224D002C34CF0530E4C6223
:101770001FD003C34CF0570E4C621AD005C34CF077
:101780003B0E4C6215D004C37CF07C6702D0300E57
:101790007C6F310E7C6305D07AC0C7F17BC0C8F185
:1017A00007D0300E7C6304D078C0C7F179C0C8F18F
:1017B000346ADBEF0BF00880140E2A6E1200140E50
:1017C00096EC0DF0C7EC16F078C04CF079C04DF0F7
:1017D0001BEC21F026EC20F0540E96EC0DF0C7EC3B
:1017E00016F07AC04CF07BC04DF01BEC21F026ECDB
:1017F00020F0400E96EC0DF07C5109EC0DF008EC59
:101800000CF0120006EC0CF008EC0CF008EC0CF0FC
:101810000EEC0CF00EEC0CF00EEC0CF0FA0E12D0FC
:10182000C80E10D0640E0ED0320E0CD01E0E0AD090
:101830000A0E08D0050E06D0030E04D0020E02D008
:10184000010E00D00B6E060E0A6EF80E096E092E00
:10185000FED70A2EFCD70B2EF6D712000F01806A96
:10186000896A000E386F1F0E926E816A8A6A000EB6
:10187000396F010E936E826A8B6A800E946E000E31
:101880003A6F836A8C6A000E956E000E3B6F846A15
:101890008D6A000E3C6F070E966E000EC16EBE0E76
:1018A000C06E000ED06EC00EF26E400EF16E000ED5
:1018B000F06E010E9D6E000EA06E220ED56E130E00
:1018C000CD6E000EBA6E000EB16E0001010E816E7B
:1018D000F00E826E000E836E070E846E11D8000E1D
:1018E000CE6E4C0ECF6E05EE00F015EE00F0EACF96
:1018F00083F0E9CF82F0E2CF85F0E1CF84F01200EF
:10190000716B00EE00F0EE6A712FFDD7040E726F5E
:1019100001EE00F0EE6A712FFDD7722FFBD7120097
:1019200080A61200809A8392839014EC0CF0200E13
:1019300069EC0DF0800E69EC0DF018EC0CF0200E47
:1019400069EC0DF0800E69EC0DF020EC0CF0060E49
:101950005BEC0DF00C0E5BEC0DF0140E5BEC0DF07F
:1019600029EC0DF0B6EC0CF08EEF0DF08EEC0DF0D6
:10197000000EF86E2C0EF76E940EF66EAAEC0DF0BB
:10198000000EF86E2C0EF76EAA0EF66EAAEC0DF095
:10199000000EF86E2C0EF76EC00EF66EAAEC0DF06F
:1019A000000E356208D0000EF86E2C0EF76ED60EC3
:1019B000F66EAAEC0DF0010E356208D0000EF86E3E
:1019C0002C0EF76EEC0EF66EAAEC0DF0030E3562DF
:1019D00008D0000EF86E2C0EF76EF80EF66EAAEC1C
:1019E0000DF0040E356208D0000EF86E2D0EF76E65
:1019F0000A0EF66EAAEC0DF0020E356208D0000E4B
:101A0000F86E2D0EF76E1C0EF66EAAEC0DF006EFBA
:101A10000CF03C6E79EC0DF03C5083828390809A00
:101A2000F00B69EC0DF03C38F00B53D03C6E3C46AB
:101A30003C463C4679EC0DF03C5040095BEC0DF027
:101A4000080E716F0900F55009EC0DF0712FFAD7EF
:101A5000120080A61200000EF86E1A0EF76E760EB7
:101A6000F66E080E726F736B735116EC0DF0732BDC
:101A7000722FFAD7120000000E11110A1B0000008D
:101A800010101000011500001414140001150000BE
:101A90001515150001150E1111110A0A1B00000081
:101AA0000000000000000000000000000000000036
:101AB00000000000000080A612003C6E79EC0DF0E2
:101AC0003C50F00B83928390809A69EC0DF03C3887
:101AD000F00B80A61200E8380F0B82B8100982BA0A
:101AE000200982BC400982BE8009826E808A809A69
:101AF000120080A6120082869486839283806E975D
:101B0000808A000082A66E87809A0000808A00008A
:101B1000809A6EA7F4D7949683901200010ECBD7CB
:101B2000020EC9D7800EC7D7C00EC5D78009C3D74C
:101B3000200E6FD7716F98EC0DF0712FFCD712004B
:101B40003D6E3D380EEC00F009EC0DF03D500EEC12
:101B500000F05FD70900F55096EC0DF00900F55044
:101B600003E009EC0DF0FAD71200BEEC0DF01FEC0B
:101B70000EF002E0D88001D0D89012008B808B82CA
:101B80008B848B8612008B908B928B948B96120099
:101B9000B5EC0DF0FDE30C6AFBEC0DF00C6E040EE1
:101BA000716F18EC0CF0FBEC0DF00C62F1D7712F9B
:101BB000F8D7000E0CB807D0030E0CBA04D0060EEE
:101BC0000CBC01D0090E726F010E0CB404D0020ED1
:101BD0000CB201D0030E722772C00CF0500E716F60
:101BE000B5EC0DF006E318EC0CF0712FF9D7100EE0
:101BF0000C262D681200C3EC0DF08B801FEC0EF04C
:101C000015E1C3EC0DF08B821FEC0EF00FE1C3EC7D
:101C10000DF08B841FEC0EF009E1C3EC0DF08B8608
:101C20001FEC0EF003E1726BE86A12008250E83894
:101C3000F00B726F1FEC0EF07211C3EF0DF08450B9
:101C4000070BE8A002D0040E02D0E8B4010E120087
:101C50000C6AB5EC0DF0FCE31200B5EC0DF0FDE202
:101C600012001D0E0DD0190E0BD0150E09D0110E3D
:101C700007D00D0E05D0090E03D0050E01D0010EC0
:101C8000C26EC282C2B2FED7C4CF77F0C3CF76F0A5
:101C90001200A6B2FED705C0A9FF06C0A8FFA69EE7
:101CA000A69CA684F29EF2BEFDD7550EA76EAA0E84
:101CB000A76EA68207A4F28EA6941200A6B2FED743
:101CC00005C0A9FFA69EA69CA680A8CF06F012007C
:101CD000DECF06F049EC0EF0052A712FF9D712007D
:101CE0005EEC0EF006C0DEFF052A712FF9D7120058
:101CF000410E90EC0EF0490E90EC0EF0320E90EC8E
:101D00000EF03B0E0DD0030E356202D03B0E01D01B
:101D10001D0EAF6EAC94AC8AAB88AB8E9D8A120060
:101D20009EA8FED7AD6E120084C0E1FF85C0E2FF21
:101D30008251E15C02E1D8901200E650326EF10E61
:101D4000E15C02E115EE00F0E1CF84F0E2CF85F036
:101D50003250D8801200010E356207D0346A040E6A
:101D6000716F09D8030E90EF0EF01200010E35626C
:101D700007D0050E716FE86A90EC0EF0712FFBD75B
:101D80001200056A5EEC0EF006C035F0120035C098
:101D900006F0056A49EC0EF012EF0CF0910E0D62A0
:101DA00003D0000E356E2CD0920E0D6203D0010EC2
:101DB000356E26D0930E0D6203D0020E356E20D004
:101DC000940E0D6203D0030E356E1AD0950E0D627F
:101DD00003D0040E356E14D08B0E0D6202D003EFCB
:101DE0000FF0810E0D6202D042EF0FF0710E0D6206
:101DF00002D081EF0FF0720E0D6202D0ACEF0FF047
:101E0000C6DF078212007C6B8EEC0DF00C6A0D6A47
:101E1000B5EC0DF00CE3C8EC0DF00C0E0C6201D02B
:101E2000FF000B0E0C6203D08EEC0DF07C6B94EC7B
:101E30000EF0ECE3280E7C6301D07C6B7C6705D050
:101E400073EC13F0000E96EC0DF00A0E7C6305D0D7
:101E50007CEC13F0400E96EC0DF0140E7C6305D074
:101E600085EC13F0140E96EC0DF01E0E7C6305D07D
:101E70008EEC13F0540E96EC0DF03250A0EC0DF0F9
:101E80007C2BC4D77C6B8EEC0DF00C6A0D6AB5EC24
:101E90000DF00CE3C8EC0DF00C0E0C6201D0FF004D
:101EA0000B0E0C6203D08EEC0DF07C6B94EC0EF0FC
:101EB000ECE3500E7C6301D07C6B7C6705D073EC47
:101EC00013F0000E96EC0DF0140E7C6305D07CEC44
:101ED00013F0400E96EC0DF0280E7C6305D085ECD7
:101EE00013F0140E96EC0DF03C0E7C6305D08EECD6
:101EF00013F0540E96EC0DF0325009EC0DF07C2BE3
:101F0000C4D77C6B8EEC0DF0000EF86E290EF76EC8
:101F1000340EF66EAAEC0DF00C6A0D6AB5EC0DF0FD
:101F20001AE3C8EC0DF01C0E0C6201D0FF000A0E83
:101F30000C6202D02A0E0DD00B0E0C6202D0300EB5
:101F400008D00C0E0C6202D0230E03D00CC0E8FFA8
:101F5000300909EC0DF0E0D77C6B8EEC0DF0000E33
:101F6000F86E290EF76E340EF66EAAEC0DF0000E28
:101F7000F86E290EF76E600EF66EAAEC0DF00C6A84
:101F80000D6AB5EC0DF056E3C8EC0DF01C0E0C62BA
:101F900001D0FF000C0E0C624DD08EEC0DF0000E47
:101FA000F86E290EF76E4A0EF66EAAEC0DF008ECEC
:101FB0000CF08EEC0DF085EC02F08EEC0DF012EED4
:101FC0000CF00A0E716FE6CFE8FFA0EC0DF0712F58
:101FD000FAD7090E716F400E96EC0DF0E6CFE8FFD0
:101FE000A0EC0DF0712FFAD707BC09D0000EF86EE7
:101FF000290EF76E760EF66EAAEC0DF008D0000EE4
:10200000F86E290EF76E8C0EF66EAAEC0DF006EC4B
:102010000CF0000EF86E290EF76E340EF66EAAEC78
:102020000DF0000EF86E290EF76E600EF66EAAEC3B
:102030000DF000D0A4D7F8EC12F02DEC12F0B9ECB2
:1020400016F0C5C14CF0C6C14DF04C5204E14D52E2
:1020500002E12CEF12F03CEC19F0B3EC1AF0FBECBF
:102060001CF049EC1BF0ECEC1CF0C9EC1AF0CEECC7
:102070001CF0C9EC1AF061C02CF162C02DF163C0F4
:102080002EF164C02FF165C030F100C261F001C2D1
:1020900062F002C263F003C264F004C265F02CC1B6
:1020A00066F02DC167F02EC168F02FC169F030C114
:1020B0006AF0C9EC1AF061C091F162C092F163C09C
:1020C00093F164C094F165C095F105C261F006C258
:1020D00062F007C263F008C264F009C265F02CC167
:1020E00066F02DC167F02EC168F02FC169F030C1D4
:1020F0006AF0C9EC1AF061C022F162C023F163C03A
:1021000024F164C025F165C026F11DEC1DF0F0EC52
:1021100016F022C166F023C167F024C168F025C122
:1021200069F026C16AF049EC1BF0658F61C096F139
:1021300062C097F163C098F164C099F165C09AF1EB
:10214000010E1A6231D0C6EC1CF066C04BF167C0BC
:102150004CF168C04DF169C04EF16AC04FF191C1B8
:1021600050F192C151F193C152F194C153F195C113
:1021700054F1616B626B636B646B656B61C055F1AD
:1021800062C056F163C057F164C058F165C059F19F
:1021900096C15AF197C15BF198C15CF199C15DF1AB
:1021A0009AC15EF1C6EC28F0020E1A6244D0616B4F
:1021B000626B636B646B656B61C050F162C051F11F
:1021C00063C052F164C053F165C054F161C055F170
:1021D00062C056F163C057F164C058F165C059F14F
:1021E000C6EC1CF066C04BF167C04CF168C04DF105
:1021F00069C04EF16AC04FF196C15AF197C15BF1C7
:1022000098C15CF199C15DF19AC15EF1C6EC28F00C
:102210000101556B566B576B586B596B000191C19F
:102220005AF192C15BF193C15CF194C15DF195C12A
:102230005EF130EC26F0030E1A6231D0C6EC1CF0D1
:1022400066C04BF167C04CF168C04DF169C04EF1FA
:102250006AC04FF196C150F197C151F198C152F146
:1022600099C153F19AC154F1616B626B636B646BFA
:10227000656B61C055F162C056F163C057F164C02F
:1022800058F165C059F191C15AF192C15BF193C106
:102290005CF194C15DF195C15EF1C6EC28F0040ECD
:1022A0001A6244D0616B626B636B646B656B61C077
:1022B00050F162C051F163C052F164C053F165C086
:1022C00054F161C055F162C056F163C057F164C06A
:1022D00058F165C059F1C6EC1CF066C04BF167C0FF
:1022E0004CF168C04DF169C04EF16AC04FF191C127
:1022F0005AF192C15BF193C15CF194C15DF195C15A
:102300005EF1C6EC28F00101556B566B576B586BAC
:10231000596B000196C15AF197C15BF198C15CF10C
:1023200099C15DF19AC15EF130EC26F01A6616D0C3
:10233000C6EC1CF066C04BF167C04CF168C04DF1B3
:1023400069C04EF16AC04FF191C150F192C151F193
:1023500093C152F194C153F195C154F1050E1A6223
:1023600016D0C6EC1CF066C04BF167C04CF168C0DB
:102370004DF169C04EF16AC04FF196C150F197C15D
:1023800051F198C152F199C153F19AC154F101012F
:10239000547F00014BC19BF14CC19CF14DC19DF19B
:1023A0004EC19EF14FC19FF150C1A0F151C1A1F1A9
:1023B00052C1A2F153C1A3F154C1A4F14BC161F0C8
:1023C0004CC162F04DC163F04EC164F04FC165F085
:1023D0004BC166F04CC167F04DC168F04EC169F069
:1023E0004FC16AF0C9EC1AF061C00EF162C00FF182
:1023F00063C010F164C011F165C012F150C161F009
:1024000051C162F052C163F053C164F054C165F030
:1024100050C166F051C167F052C168F053C169F014
:1024200054C16AF0C9EC1AF00EC166F00FC167F032
:1024300010C168F011C169F012C16AF08CEC1BF098
:10244000F5EC1BF061C0A5F162C0A6F163C0A7F175
:1024500064C0A8F165C0A9F11200B9EC16F01CC067
:102460004CF01DC04DF03CEC19F0B3EC1AF006EC4A
:1024700017F01CC04CF01DC04DF0640E516E000EE4
:10248000526E52504D5C02E151504C5CD8B001D0BC
:102490008DD0C80E516E000E526E52504D5C02E14E
:1024A00051504C5CD8B001D054D02C0E516E010E5E
:1024B000526E52504D5C02E151504C5CD8B001D08C
:1024C00048D0900E516E010E526E52504D5C02E19A
:1024D00051504C5CD8B001D03CD0F40E516E010E7E
:1024E000526E52504D5C02E151504C5CD8B001D05C
:1024F00030D0580E516E020E526E52504D5C02E1B9
:1025000051504C5CD8B001D024D0BC0E516E020E9C
:10251000526E52504D5C02E151504C5CD8B001D02B
:1025200018D0200E516E030E526E52504D5C02E1D7
:1025300051504C5CD8B001D00CD0840E516E030EBB
:10254000526E52504D5C02E151504C5CD8B001D0FB
:1025500000D0C7EC16F051C04CF052C04DF03CEC2E
:1025600019F0B3EC1AF0FBEC1CF086EC1BF08AECD3
:1025700017F0FBEC1CF086EC1BF095EC17F0E5EC8B
:1025800016F01CEC17F086EC1BF03F0E6A6FB30ED2
:10259000696F330E686F330E676F330E666FC9EC69
:1025A0001AF032EC17F08CEC1BF00ED0E5EC16F0C4
:1025B0003E0E6A6FBD0E696F700E686FA30E676F77
:1025C000D70E666FC9EC1AF0410E6A6F880E696FFC
:1025D000666B676B686B8CEC1BF061C005F262C0C8
:1025E00006F263C007F264C008F265C009F2120087
:1025F000B9EC16F01BC04CF03CEC19F0B3EC1AF03F
:102600003E0E6A6F666B676B686B696BC9EC1AF09C
:1026100061C000F262C001F263C002F264C003F262
:1026200065C004F21200EACF04F0E9CF03F083C0E2
:10263000EAFF82C0E9FF9EAA0ED0AE50ABA204D042
:10264000AE50AB98AB88F7D7EE6EF10EE95C02E1C5
:1026500005EE00F0F0D7EACF83F0E9CF82F0F2A4E4
:1026600002D0F29430D0F2A202D0F2922CD09EA0EE
:1026700022D09E9022662206236623062466240624
:102680002566250626662606286602D0275206E01D
:1026900027062728D8B42806D8B427522966290641
:1026A0002A662A062B662B062C662C06000ECE6E9A
:1026B0004C0ECF6E08D0A1A802D0A19804D09EA243
:1026C00002D09E9200D004C0EAFF03C0E9FF1100CF
:1026D000006ED8CF01F0E0CF02F002C0E0FF005062
:1026E00001C0D8FF1000000EF86E270EF76E2E0EF8
:1026F000F66EAAEC0DF01200000EF86E270EF76EC3
:10270000440EF66EAAEC0DF01200000EF86E270EC5
:10271000F76E5A0EF66EAAEC0DF01200000EF86E6F
:10272000270EF76E700EF66EAAEC0DF01200002068
:102730002020202020202020202020202020202099
:102740002020200040202020202020202020202089
:1027500020202020202020202000142020202020A5
:102760002020202020202020202020202020200089
:102770005420202020202020202020202020202025
:102780002020202020000B505374617200000B4663
:102790005438343700000B4B3220202000000B50FF
:1027A0007753445200000A49433733303000004326
:1027B0003A00404C3A000A433A004A4C3A00144965
:1027C0006D706564616E7A3D2000545A3D200000B2
:1027D00014503A0054463A0054663A0011413A0007
:1027E0004B5357523A002043524320213D00062DBF
:1027F0004C2D0000462020200000062D4C2B000010
:10280000462020430000062B4C2D0000464320208C
:102810000000062D432B00004620204C0000062B14
:10282000432D0000464C20200000062D432D0000C3
:102830004620202000004D487A006B487A007548F9
:102840000000704600000042656665686C3A200032
:10285000005452582052656D6F74653A203900005B
:10286000405B315D5069636153746172205B345D1C
:102870004B3220202000145B325D46543834372020
:102880002020205B355D507753445200545B335D0C
:1028900049433733303020202020202020202020A2
:1028A0000000005253323332204D6F6E69746F72E4
:1028B0003A203800405B305D2048657864657A696D
:1028C0006D616C20202020202000145B315D2041B0
:1028D00073636369202020202020202020202000F6
:1028E000545B235D20416262727563682020202062
:1028F0002020202020000054657366756E6B74697B
:102900006F6E656E3A203700405B315D2054617315
:1029100074656E66656C6420202020202000145BA6
:10292000325D204C45442D446174656E7472616E55
:1029300073662E00545B23206C616E675D204162DC
:102940006272756368212120200000446174656E05
:102950006162727566202D2D2D3E202020202000E2
:10296000145B235D20446174656E6162727566203C
:10297000202020202000143D3D3D3D206572666FE3
:102980006C677265696368203D3D3D00143D3D3DC7
:102990003D206665686C657268616674203D3D3DEA
:1029A0003D00003D204B65696E6520446174656E95
:1029B00020766F6D203D2000403D20416E74656E95
:1029C0006E656E2D54756E657221203D2000143D9C
:1029D0002057617274656E20352053656B2120206D
:1029E000203D2000543D20566572737563683A207F
:1029F0003D200000543D20776569746572206D6943
:102A0000742022232220203D20001F435243206FA8
:102A10006B2100001F43524320213D200000003D58
:102A20003D3D3D2053796D54756E6572203D3D3DB1
:102A30003D3D2000403D3D20696D20536C65657033
:102A40006D6F647573203D3D3D00003D3D3D3D3D56
:102A50002046756E6B74696F6E203D3D3D3D3D00B7
:102A6000402D2D2053706569636865726E20426148
:102A70006E64202D2D00402D537065692E31306B12
:102A8000487A205365676D656E742D00402D2D2D9D
:102A90002D204E61636874756E656E202D2D2D2D71
:102AA0002D00142D2062697320535752204D696EFA
:102AB000696D756D202D2D00402D2054756E656E4D
:102AC00020696E20466C6165636865202D00142DB9
:102AD0002D2D206269732053575220312C00232062
:102AE0002D2D2D2D0000142D2D20696E20466C619A
:102AF0006563686520387838202D2D00542D2D2DE4
:102B00002D2054756E656E20617573202D2D2D2D31
:102B10002D00542D2D2057617274656E205458205D
:102B20004F4E202D2D2D2D00542D2D2057617274C8
:102B3000656E205458204F4646202D2D2D00402DE7
:102B40002D416E74656E6E65206C6F65736368658C
:102B50006E2D2D00402D205049436565202D2D3EC2
:102B6000206578746565202D2D00402D20657874D2
:102B70006565202D2D3E205049436565202D2D0093
:102B8000402D20506F7765722C2053575220434CB4
:102B900052202D2D2D00402D2D2D204657205665DD
:102BA0007273696F6E656E202D2D2D001454756E35
:102BB0006572203A00005452656D6F74653A0000EA
:102BC000142057617274656E20626973204C45440D
:102BD000206175732100542057617274656E206204
:102BE0006973204C4544206175732100162D2D3EDC
:102BF0002000402D2D416E74656E6E65206B6F70E8
:102C0000696572656E2D2D0014205B395D204F4B78
:102C100020576569746572202020202020005420F0
:102C20005B235D2041626272756368202020202052
:102C300020202000004265662E34362077696564C6
:102C40006572686F6C656E21200040437765727411
:102C50003D0014696E20746965666572656E204278
:102C6000657265696368200014696E20686F656825
:102C70006572656E20426572656963682000546DF7
:102C80006974204265662E34332077656368736506
:102C90006C6E21000053796D54756E65722044543A
:102CA0004D462D52656D6F746500404857312E308A
:102CB0003220202032302E31312E3230323120007D
:102CC000145357322E31312D34354B3232202044BB
:102CD0004C344A414C00544341542D506963415394
:102CE00074617220444C344A414C20005443415496
:102CF0002D46542038343700544341542D4B322054
:102D0000456C6563726166740000544341542D50F4
:102D1000432D506F77657253445200005443415421
:102D20002D4943373330302049636F6D00002D2D1E
:102D30002D00494E46006D570000755700006E5734
:102D400000007057000066570000615700005720D0
:102D500000006B570000205600006D5600007556AD
:102D600000006E56000064426D0064420000737300
:102D7000000013D806D8476A486A496A4A6A4B6A0B
:102D80001200426A436A446A456A466A12004C6A03
:102D90004D6A4E6A4F6A506A1200F9DF516A526AF0
:102DA000536A546A556A1200616B626B636B646BA1
:102DB000656B12000EC166F00FC167F010C168F0BC
:102DC00011C169F012C16AF012000EC161F00FC1A9
:102DD00062F010C163F011C164F012C165F012001D
:102DE00066C061F067C062F068C063F069C064F0FB
:102DF0006AC065F0120061C066F062C067F063C02F
:102E000068F064C069F065C06AF0120061C00EF13C
:102E100062C00FF163C010F164C011F165C012F11E
:102E2000120013C161F014C162F015C163F016C144
:102E300064F017C165F0120013C166F014C167F0A9
:102E400015C168F016C169F017C16AF0120018C107
:102E500061F019C162F01AC163F01BC164F01CC1BA
:102E600065F0120018C166F019C167F01AC168F068
:102E70001BC169F01CC16AF012001DC161F01EC1C6
:102E800062F01FC163F020C164F021C165F012003F
:102E90001DC166F01EC167F01FC168F020C169F056
:102EA00021C16AF0120022C161F023C162F024C185
:102EB00063F025C164F026C165F0120022C166F0FE
:102EC00023C167F024C168F025C169F026C16AF00A
:102ED000120027C161F028C162F029C163F02AC144
:102EE00064F02BC165F0120027C166F028C167F0BD
:102EF00029C168F02AC169F02BC16AF0120066C0CE
:102F000013F167C014F168C015F169C016F16AC009
:102F100017F1120061C013F162C014F163C015F122
:102F200064C016F165C017F1120061C018F162C0EB
:102F300019F163C01AF164C01BF165C01CF11200E5
:102F400061C01DF162C01EF163C01FF164C020F1B9
:102F500065C021F1120061C022F162C023F163C09B
:102F600024F164C025F165C026F1120061C027F18B
:102F700062C028F163C029F164C02AF165C02BF159
:102F8000120042C04CF043C04DF044C04EF045C06A
:102F90004FF046C050F0120042C051F043C052F012
:102FA00044C053F045C054F046C055F012004CC028
:102FB00042F04DC043F04EC044F04FC045F050C009
:102FC00046F01200513652365336543655361200FA
:102FD0004C364D364E364F3650361200553254323E
:102FE000533252325132120050324F324E324D3241
:102FF0004C32120006D84736483649364A364B36E8
:1030000012004236433644364536463612004B32BD
:103010004A324932483247321200F9DF46324532ED
:1030200044324332423212004CAE04D04D684E68F6
:103030004F68506812004DAE03D04E684F6850681C
:1030400012004EAE02D04F68506812004FAE01D051
:10305000506812006F936EBF6F838CDE280E3F6E38
:10306000D890F4EC17F00EEC18F003D83F2EF8D7F8
:103070001200FDEC21F00A0E3E6E00EE42F0EF5021
:10308000E8B6FD0FE8BED00FEE6E3E2EF8D70AEC84
:1030900022F012003FD846AE09D0472AD8B4482AB9
:1030A000D8B4492AD8B44A2AD8B44B2AC1EC16F06D
:1030B00035D030D846AE09D0472AD8B4482AD8B43B
:1030C000492AD8B44A2AD8B44B2A47C042F048C04B
:1030D00043F049C044F04AC045F04BC046F06EBFD3
:1030E00002EC1FF0120016D847C042F048C043F06F
:1030F00049C044F04AC045F04BC046F06EBF02ECF8
:103100001FF0120007D8BBEC16F008D003D8C1ECB2
:1031100016F004D09DEC1AF092EF18F04FEC19F075
:10312000B3EF1AF04CD803E1BAEC16F01AD01AD863
:103130007F0E566E56505A5E57505B5A5AC03EF03C
:103140005A520FE05ABE06D0D890FAEC17F03E2E35
:10315000FBD707D03E1E3E2AD8900DEC18F03E2E2D
:10316000FBD712006E9F60BF6E8F609FBAEC16F0A7
:103170005CC043F05DC044F05EC045F05FC046F007
:1031800060C047F0D890FAEC17F00EEC18F0468EBD
:1031900047C05AF0476AD890FAEC17F01200040EB4
:1031A0003E6EEE6608D03E2EFCD7EECFE8FF7F0BDA
:1031B00003E1D88401D0D8940AEC22F01200FDEC8F
:1031C00021F000EE5CF0EBD7FDEC21F000EE61F0B9
:1031D000E6D7FDEC21F000EE66F0E1D7FDEC21F042
:1031E00000EE4CF0DCD7FDEC21F000EE51F0D7D72B
:1031F000FDEC21F000EE42F00A0E3E6EEE66DBD7EB
:103200003E2EFCD7D6D7506A4FBE506835D04F6A95
:10321000506A4EAE31D04F6850682ED04E6A4F6A19
:10322000506A4DAE29D04E684F68506825D04D6A1F
:103230004E6A4F6A506A4CAE1FD04D684E684F6858
:1032400050681AD0BAEC16F06E9F506A1DD0BAECD6
:1032500016F06E9F4F6A506A17D0BAEC16F06E9F48
:103260004E6A4F6A506A10D0BAEC16F06E9F4D6AE3
:103270004E6A4F6A506A08D0BAEC16F06E9F50AE94
:1032800003D011EC1FF06E8F4CC047F04DC048F0DA
:103290004EC049F04FC04AF050C04BF000D07F0EF6
:1032A0005A6E000E5B6EF8EC18F006E15C6A5D6A1F
:1032B0005E6A5F6A606B36D0B9EC19F007E0D890AF
:1032C0000DEC18F05A2AD8B45B2AF6D747B00AD0CA
:1032D000D890FAEC17F05A065A28D8B45B06D8B43E
:1032E0005A52F4D743A00BD04380432AD8B4442A7F
:1032F000D8B4452AD8B4462AD8B4472ADDD7426A7A
:1033000047905AC047F00DEC18F043C05CF044C041
:103310005DF045C05EF046C05FF047C060F0609F62
:103320006EBF608F12005C6A5D6A5E6A606B800EC1
:103330005F6EF5D75C685D685E687F0E5F6E7F0EBE
:10334000606FEDD77F0E4C6E000E4D6E5B504D5C86
:1033500002E15A504C5CD8B003D0ECDFD88401D0E5
:10336000D89412005BAE03D0DEDFD88401D0D894AD
:103370001200FDEC21F000EE4BF0040E3E6EED6607
:103380000AD03E2EFCD7010EEF6201D002D0EF66CC
:1033900002D0D88401D0D8940AEC22F0120051C097
:1033A00000F152C001F153C002F154C003F155C005
:1033B00004F119EC1AF042C007F143C008F144C00F
:1033C00009F145C00AF146C00BF100C14CF001C142
:1033D0004DF002C14EF003C14FF004C150F0FFECBC
:1033E00019F007C147F008C148F009C149F00AC106
:1033F0004AF00BC14BF06E9F6FB36E8F1200BADCB8
:10340000280E3F6ED89005D801EC18F03F2EFAD761
:103410001200FDEC21F0050E3E6E00EE4CF0D8904F
:10342000EF50E8200700EE6E3E2EFAD70AEC22F0AD
:103430001200FDEC21F09EDC280E3F6ED890F4ECDB
:1034400017F00EEC18F000EE4CF0050E3E6EEFAEED
:1034500002D0300EEF5EEFA602D0030EEF5EEE520A
:103460003E2EF5D73F2EEAD70AEC22F0120002D802
:10347000C1EF17F0FDEC21F09ADD00EE42F010EE06
:1034800051F0040E3E6EE650EE5EE650EE5A3E2ED1
:10349000FCD70AEC22F0120002D8C1EF17F0FDECC5
:1034A00021F085DD00EE42F010EE51F0E650EE2600
:1034B000040E3E6EE650EE223E2EFCD70AEC22F0C1
:1034C000120000C14CF001C14DF002C14EF003C129
:1034D0004FF004C150F005C156F006C157F012007C
:1034E00007C151F008C152F009C153F00AC154F0AC
:1034F0000BC155F00CC158F00DC159F0120043C07A
:1035000000F144C001F145C002F146C003F147C0DB
:1035100004F15AC005F15BC006F1120043C007F187
:1035200044C008F145C009F146C00AF147C00BF19B
:103530005AC00CF15BC00DF1120061C05CF062C0BA
:103540005DF063C05EF064C05FF065C060F01200C3
:1035500066C05CF067C05DF068C05EF069C05FF097
:103560006AC060F012005CC061F05DC062F05EC0D5
:1035700063F05FC064F060C065F012005CC066F08C
:103580005DC067F05EC068F05FC069F060C06AF05F
:1035900012001AEC22F016E217EC22F013E2E4EC2F
:1035A00018F01AE0E9EC18F017E02FEC22F004E331
:1035B000E4EC18F001E306D032EC22F006E3E9EC8B
:1035C00018F003E357EC22F012002FEC22F003E393
:1035D0004CEC22F003D00DD0D4EC16F065BF03D034
:1035E0006AAF01D0658F65AF03D06ABF01D0658F28
:1035F00012001DD86E9F6EBB6E7F6EBD6E7FBEECDF
:103600001EF046C000F147C001F148C002F149C0B8
:1036100003F14AC004F11ED84FEC1AF0C1EC17F0C8
:10362000CEEC16F07F0E516E3AEC1AF01ED06E9B67
:103630006E9D65BF6E8B6ABF6E8D7FDFB2EC18F03A
:103640005EDF86DFB2EC18F069DFB9EC16F039DF27
:1036500070EF1AF0B9EC16F056C04CF057C04DF0B0
:1036600058C051F059C052F0120042C05AF043C045
:103670005BF0BAEC16F000C143F001C144F002C1A6
:1036800045F003C146F004C147F053EC19F0B3EF25
:103690001AF01AEC22F009E217EC22F006E2E4EC50
:1036A00018F006E1E9EC18F019E157EC22F01200ED
:1036B00032EC22F003E32FEC22F0F7E2E9EC18F011
:1036C00010E14CEC22F065BF03D06AAF01D0658FEA
:1036D00065AF03D06ABF01D0658F120061EC22F0A4
:1036E000F2D7A5DF6E9F6EBB6E7F6EBD6E7F8CECDA
:1036F0001FF005DFAFDF3AEC1AF0C1EC17F0CEECAB
:1037000016F07F0E516E4FEC1AF0AFD7E9EC18F0BF
:1037100001E112006A7F00D01AEC22F004E217ECFB
:1037200022F001E203D057EC22F01200E9EC18F08D
:1037300001E11200E4EC18F003E1F0EC16F01200E5
:1037400017D84FEC1AF056C05AF057C05BF06E9F76
:1037500046AE03D06E8F02EC1FF042C000F143C0B2
:1037600001F144C002F145C003F146C004F181D724
:103770005EDFFE0E5A6E000E5B6E5950575C02E122
:103780005850565C27E013E3582AD8B4592A5B50A6
:10379000595C02E15A50585C07E1CEEC16F056C075
:1037A00058F057C059F016D0D89018DCE6D7562AF2
:1037B000D8B4572A5B50575C02E15A50565C07E177
:1037C000C7EC16F058C056F059C057F003D0D89047
:1037D0000BDCD3D76EBB11EC1FF06EBD20EC1FF0DD
:1037E0001200FBEC16F0C9EF1AF0E4EC18F02DE033
:1037F00065BF2CD01AEC22F028E206EC17F0ECD8CA
:1038000048DF8AEC17F01E0E416E414E1ED0E5ECEB
:1038100016F01CEC17F03DDF1CEC17F07DDFDCD858
:1038200038DF1CEC17F06A51655D0BE16951645D8E
:1038300008E16851635D05E16751625D02E166512F
:10384000615D03E08AEC17F0E0D7120057EC22F03C
:103850001200E4EC18F008E13F0E656F800E646F13
:10386000616B626B636B120001013F0E266F800E6D
:10387000256F226B236B246B3F0E216F800E206F10
:103880001D6B1E6B1F6B000195EC17F08AEC17F097
:1038900022C10EF123C10FF124C110F125C111F194
:1038A00026C112F11E0E416E11EC17F048EC17F014
:1038B000F0DEDAEC16F08CEC1BF0DAEC16F06A5164
:1038C000655D0BE16951645D08E16851635D05E187
:1038D0006751625D02E16651615D17E0414E15D0AE
:1038E00006EC17F053EC17F06FD816DFABEC17F0BF
:1038F00048EC17F04EDEA0EC17F027EC17F01CECAC
:1039000017F047DE8AEC17F0CFD71200E4EC18F07E
:1039100008E13F0E656F800E646F616B626B636BD5
:10392000120061C02CF162C02DF163C02EF164C0A1
:103930002FF165C030F182EC18F03BD82ADE89DF28
:10394000B6EC17F02CC161F02DC162F02EC163F00E
:103950002FC164F030C165F08AEC18F06E956EBF2F
:103960006E8547C041F027C161F028C162F029C1CE
:1039700063F02AC164F02BC165F0415206E06EA5E8
:10398000C5D86EB5D5D8412EFAD71200420E6A6F4F
:10399000480E696F666B676B686B1200400E6A6F4A
:1039A000490E696F0F0E686FDA0E676FA20E666FB1
:1039B0001200400E6A6F130E696F5D0E686F8D0EF8
:1039C000676FDE0E666F12003F0E6A6F800E696FC2
:1039D000666B676B686B1200400E6A6F666B676B95
:1039E000686B696B1200410E6A6F200E696F666B1F
:1039F000676B686B1200420E6A6FC80E696F666B68
:103A0000676B686B1200440E6A6F7A0E696F666BA3
:103A1000676B686B1200460E6A6F1C0E696F400E72
:103A2000686F666B676B1200470E6A6FC30E696F33
:103A3000500E686F666B676B1200490E6A6F740EEA
:103A4000696F240E686F666B676B12004B0E6A6FAE
:103A5000180E696F960E686F800E676F666B1200A6
:103A60004C0E6A6FBE0E696FBC0E686F200E676FDA
:103A7000666B12004E0E6A6F6E0E696F6B0E686F8A
:103A8000280E676F666B12003D0E6A6FCC0E696F71
:103A9000CC0E686FCC0E676FCD0E666F12003C0EB9
:103AA0006A6F230E696FD70E686F0A0E676F3D0E3F
:103AB000666F12003A0E6A6F830E696F120E686F9E
:103AC0006E0E676F980E666F1200350E6A6F860E67
:103AD000696F370E686FBD0E676F060E666F120056
:103AE000300E6A6F890E696F700E686F5F0E676FB8
:103AF000410E666F12002B0E6A6F8C0E696FBC0E42
:103B0000686FCC0E676F090E666F12006CDFC9EF2D
:103B10001AF071DFC9EF1AF076DFC9EF1AF07BDF18
:103B2000C9EF1AF081DFC9EF1AF087DFC9EF1AF089
:103B30005ADF49EF1BF05FDF49EF1BF064DF49EF0D
:103B40001BF069DF49EF1BF06FDF49EF1BF075DFFA
:103B500049EF1BF0E4EC18F003E157EC22F01200FF
:103B600006EC17F001013F0E176F800E166F136BF6
:103B7000146B156B000128DF86EC1BF095EC17F039
:103B8000E5EC16F021DF8CEC1BF0A0EC17F027EC35
:103B900017F048EC17F049EC1BF095EC17F0ABEC84
:103BA00017F006EC17F0280E416E11EC17F014DF39
:103BB0008CEC1BF08AEC17F027EC17F05EEC17F09A
:103BC000C9EC1AF05EEC17F0C9EC1AF095EC17F09E
:103BD0001CEC17F049EC1BF0DAEC16F08CEC1BF047
:103BE000DAEC16F06A51655D0BE16951645D08E13C
:103BF0006851635D05E16751625D02E16651615D97
:103C000005E0414E03D006EC17F0CFD7E5DEC9EF53
:103C10001AF00101276B0001F3EC1CF048D806E311
:103C200098EC1DF00101272B0001F6D793DFC1DED0
:103C300049EC1BF0B9EC16F027C147F0475206E0FB
:103C40004FEC19F0BEEC1AF08CEC1BF012007ED891
:103C500050AE14D055AE29D05AD85050555C0BE117
:103C60004F50545C08E14E50535C05E14D50525C9E
:103C700002E14C50515CD8B016D017D050BE02D0E3
:103C800055BE11D044D85050555C0BE14F50545C98
:103C900008E14E50535C05E14D50525C02E14C503E
:103CA000515CD8B002D0D89001D0D88012004ED844
:103CB00050AE14D055AE29D02AD85050555C0BE1E7
:103CC0004F50545C08E14E50535C05E14D50525C3E
:103CD00002E14C50515CD8B016D017D050BE02D083
:103CE00055BE11D014D85050555C0BE14F50545C68
:103CF00008E14E50535C05E14D50525C02E14C50DE
:103D0000515CD8B002D0D88001D0D8901200E4EC39
:103D100018F003E1C7EC16F00FD0D890E8EC17F0DC
:103D2000D8904F324E324D324C324F8EE9EC18F073
:103D300003E1CEEC16F009D0D890E2EC17F0D89061
:103D40005432533252325132548E120061C04CF010
:103D500062C04DF063C04EF064C04FF065C050F0DB
:103D600066C051F067C052F068C053F069C054F0AB
:103D70006AC055F0120002D8C1EF17F0FDEC21F037
:103D800037D8050E3E6E00EE51F020EE42F0BAEC50
:103D900016F010EE4CF0050E3F6E3EC040F03F5066
:103DA000402640064006EF50E602F350DE26D9CF0B
:103DB0006BF0DACF6CF0F450DE22E86ADE22402E9F
:103DC000FCD76BC0D9FF6CC0DAFF3F2EE6D7EE52AE
:103DD00020EE42F0060E406E3E50405EDE52402E17
:103DE000FDD73E2ED6D70AEC22F06EB30BD81200C8
:103DF0006E9350AE02D015D86E7355AE02D020D857
:103E00006E731200421E431E441E451E461E422A69
:103E1000D8B4432AD8B4442AD8B4452AD8B4462AB8
:103E200012004C1E4D1E4E1E4F1E501E4C2AD8B462
:103E30004D2AD8B44E2AD8B44F2AD8B4502A1200EA
:103E4000511E521E531E541E551E512AD8B4522ABA
:103E5000D8B4532AD8B4542AD8B4552A1200C8DF8B
:103E6000FDEC21F0BAEC16F0050E3E6E00EE51F0BE
:103E7000EE6605D03E2EFCD70AEC22F012003E6A18
:103E80003E2AD89055BE1CD0513652365336543641
:103E900055365550505C0BE154504F5C08E153507F
:103EA0004E5C05E152504D5C02E151504C5CE8E241
:103EB000BAEC16F0D8905532543253325232513255
:103EC0005550505C0BE154504F5C08E153504E5C30
:103ED00005E152504D5C02E151504C5C0AE35150F7
:103EE0004C5E52504D5A53504E5A54504F5A5550A2
:103EF000505A01EC18F03E2EDDD777DF4CC051F060
:103F00004DC052F04EC053F04FC054F050C055F069
:103F1000C1EC17F00AEF22F0290E3E6EBAEC16F053
:103F20005550505C0BE154504F5C08E153504E5CCF
:103F300005E152504D5C02E151504C5C0BE3515095
:103F40004C5E52504D5A53504E5A54504F5A555041
:103F5000505AD880FAEC17F0D890E8EC17F055508A
:103F6000505C0BE154504F5C08E153504E5C05E14E
:103F700052504D5C02E151504C5C0BE351504C5E91
:103F800052504D5A53504E5A54504F5A5550505A01
:103F9000D8803E2EDFD71200FDEC21F06E9350AE9C
:103FA00002D03FDF6E83BAEC16F0280E3E6E0A0E8A
:103FB0003F6E00EE42F0EF500F0B406E050E405C7E
:103FC000D8A002D0030EEF26EF50F00B406E500E3B
:103FD000405CD8A002D0300EEF26EC523F2EEBD73B
:103FE000D890E8EC17F0FAEC17F03E2EE0D70AEC88
:103FF00022F012001AEC22F015E232EC22F01CE260
:104000002FD844D85AD86F951200030E6B6509D08B
:104010006C676B2B6EB56B2B030E6B5F6B519AEC61
:104020000DF01200F2DF000EF86E2D0EF76E2E0E60
:10403000F66EAEEC0DF01200E8DF000EF86E2D0EFD
:10404000F76E320EF66EAEEC0DF012001AEC22F0A6
:10405000E9E232EC22F0F0E203D82FD86F9512009B
:10406000FDEC21F000EE4BF011EE31F00A0E406E47
:10407000EDCF3EF03E383F6E56D83EC03FF053D8AD
:10408000402EF6D7E76A0AEC22F01200FDEC21F090
:104090006C5310E001EE44F011EE44F0140E3E6E4D
:1040A0006CC03FF0E5503E063F2EFCD7E5CFEDFF5C
:1040B0003E2EFCD70AEC22F01200FDEC21F00A0E95
:1040C0003F6E6C513F266B513F5CD8B002D03FC071
:1040D0006BF06B516C5DD8A003D06CC06BF06B2B98
:1040E0006C516B5F6B07090E3E6E6B513E5E01EECD
:1040F00031F03E5204E0EECFE8FF3E2EFCD76EA535
:1041000005D02B0E6EBF2D0ED2EC20F06E8119D88B
:104110006E9113D86C5304E02C0ED2EC20F009D829
:104120000AEC22F012003F500F0B3009E8CFE6FFF7
:1041300012006CC040F06F9706D0010E406E6F9772
:1041400002D06BC040F0405226E06EA106D0EFCF07
:104150003EF0300E3E5CD8A46E916FA711D040C0E7
:104160004CF0020E4C6202D0CCEC20F0050E4C62FA
:1041700002D0CCEC20F0080E4C6202D0CCEC20F047
:10418000EECFE8FF6EB103D0D2EC20F002D0CEEC3F
:1041900020F0402EDAD71200200E04D0200E6FB58A
:1041A000300E00D009EC0DF01200FDEC21F00A0EEB
:1041B0003E6E6C513E5E00EE42F0EF503E4E0CD033
:1041C000EF503E4E02D0EE52F8D7EE524C6E490EF2
:1041D0004C6409D0010E06D00F0B4C6E040E4C64DB
:1041E00002D0100EEF260A0E3E6E00EE42F0EF50A7
:1041F0000700EE6EE86AEF223E2EF9D70AEC22F0B5
:104200001200FDEC21F0050E3E6E0A0E3F6E00EE30
:104210004BF0EDCF4CF04C50F00B07E13F064C500B
:104220000F0B03E13F063E2EF4D73FC04CF03F504A
:104230000AEC22F0120061EC22F0BAEC16F0CCECA1
:104240001FF042C047F043C048F044C049F045C0A9
:104250004AF046C04BF0050E6B6F6C6B6E956F9518
:104260006E996F9712001AEC22F044E232EC22F0C1
:1042700041E29DEC1AF092EC18F042C000F143C00C
:1042800001F144C002F145C003F146C004F147C04A
:104290004CF048C04DF049C04EF04AC04FF04BC002
:1042A00050F0CCEC1FF042C007F143C008F144C00D
:1042B00009F145C00AF146C00BF100C14CF001C143
:1042C0004DF002C14EF003C14FF004C150F02AEC92
:1042D00018F007C147F008C148F009C149F00AC108
:1042E0004AF00BC14BF0140E6B6F0A0E6C6F6E9997
:1042F0006F976F956E95120006EC17F06D6B659FCA
:10430000E4EC18F014E0F3EC1CF057EC1EF001E0C4
:1043100004E398EC1DF06D2BF6D7E4EC1CF027ECD1
:104320001EF005E004E386EC1DF06D07F6D733ECD4
:1043300021F0E5EC16F065BF6E8F0B0E6B6F0A0E69
:104340006C6F6E856E99120026EC20F0650ED2EC33
:1043500020F06E9F6DBF6E8F6DBF6D6DC7EC16F058
:104360006DC04CF01BEC21F06E854BDF4CC06BF048
:1043700026EC20F0120011EC17F0DAEC16F086ECC7
:104380001BF0B6EC17F03DEC17F032EC17F086ECB2
:104390001BF0FBEC16F027C161F028C162F029C1C7
:1043A00063F02AC164F02BC165F049EC1BF0B6EC58
:1043B00017F053EC17F032EC17F086EC1BF074ECAE
:1043C00017F0C9EC1AF0DAEC16F08CEC1BF01200C6
:1043D000FDEC21F0C7EC16F0050E3E6E10EE42F03B
:1043E00020EE4CF0E6500F0BDF6EE638F00BDE12DD
:1043F0003E2EF8D70AEC22F01200E9CF45F1EACFC1
:1044000046F1E1CF47F1E2CF48F1D9CF49F1DACF18
:104410004AF1120045C1E9FF46C1EAFF47C1E1FF89
:1044200048C1E2FF49C1D9FF4AC1DAFF1200A8EC36
:104430001AF003D09DEC1AF000D0609F7F0E6063ED
:104440000CD0800E5F6207D05E6605D05D6603D03B
:104450005C6601D002D0D88001D0D8901200A8ECC0
:104460001AF003D09DEC1AF000D0609F7F0E6063BD
:104470000BD0800E5F6208D05E6606D05D6604D009
:104480005C6602D0D88001D0D890120002D8B3EF79
:104490001AF005D8608F120002D8B3EF1AF07F0E21
:1044A000606F800E5F6E5C6A5D6A5E6A120002D8A1
:1044B000B3EF1AF07F0E606F5C685D685E685F68DE
:1044C000120002D8B3EF1AF05C6A5D6A5E6A5F6A36
:1044D000606B1200410E6A6FA00E696F666B676BAE
:1044E000686B12006AEC22F049EC1BF086EC1CF0C1
:1044F00006EC17F0E4EC1CF08CEC1BF08AEC17F0E7
:10450000E5EC16F0E4EC1CF086EC1BF0FBEC16F08E
:1045100011EC17F049EC1BF01200AAC161F0ABC11D
:1045200062F0ACC163F0ADC164F0AEC165F098EC6F
:104530001DF086EC1CF061C0B4F162C0B5F163C03F
:10454000B6F164C0B7F165C0B8F11200B4C161F052
:10455000B5C162F0B6C163F0B7C164F0B8C165F02F
:104560009EEC1DF0C6EC1CF0C9EC1AF0F5EC1BF04B
:1045700061C0BFF162C0C0F163C0C1F164C0C2F1EB
:1045800065C0C3F11200BFC161F0C0C162F0C1C11A
:1045900063F0C2C164F0C3C165F00101010EC46FD4
:1045A000000165EC1DF027EC1EF009E30101040E8B
:1045B000C46F000195EC1DF08CEC1DF018D05AEC86
:1045C0001DF027EC1EF007E30101030EC46F00018C
:1045D00095EC1DF00CD0E4EC1CF027EC1EF007E38A
:1045E0000101020EC46F00018CEC1DF000D061C00F
:1045F000BAF162C0BBF163C0BCF164C0BDF165C07B
:10460000BEF11200B4C161F0B5C162F0B6C163F091
:10461000B7C164F0B8C165F00101030EB96F0001C4
:104620007BEC1DF027EC1EF00BE395EC1DF095ECF8
:104630001DF08CEC1DF00101080EB96F00014CD08B
:1046400070EC1DF027EC1EF009E395EC1DF095ECE5
:104650001DF00101070EB96F00013ED065EC1DF0A1
:1046600027EC1EF009E395EC1DF08CEC1DF0010128
:10467000060EB96F000130D05AEC1DF027EC1EF089
:1046800007E395EC1DF00101050EB96F000124D080
:10469000E4EC1CF027EC1EF007E38CEC1DF00101AC
:1046A000040EB96F000118D01DEC1DF057EC1EF080
:1046B00007E3A7EC1DF00101010EB96F00010CD05A
:1046C00003EC1DF057EC1EF007E39EEC1DF001011A
:1046D000020EB96F000100D061C0AFF162C0B0F14D
:1046E00063C0B1F164C0B2F165C0B3F11200AFC1F3
:1046F00061F0B0C162F0B1C163F0B2C164F0B3C1A6
:1047000065F033EC21F0050E6B6F010E6C6FF3EC6E
:104710001CF027EC1EF003E3040E6C6F0FD0FBECD3
:104720001CF027EC1EF003E3030E6C6F07D003ECC4
:104730001DF027EC1EF002E3020E6C6F67D8D5EC7B
:1047400020F026EC20F0B9C14CF0030E4C6209D0E9
:10475000000EF86E2D0EF76E360EF66EAEEC0DF006
:1047600054D0040E4C6209D0000EF86E2D0EF76E78
:104770003A0EF66EAEEC0DF048D0050E4C6209D044
:10478000000EF86E2D0EF76E3E0EF66EAEEC0DF0CE
:104790003CD0060E4C6209D0000EF86E2D0EF76E5E
:1047A000420EF66EAEEC0DF030D0070E4C6209D022
:1047B000000EF86E2D0EF76E460EF66EAEEC0DF096
:1047C00024D0020E4C6209D0000EF86E2D0EF76E4A
:1047D0004E0EF66EAEEC0DF018D0010E4C6209D004
:1047E000000EF86E2D0EF76E520EF66EAEEC0DF05A
:1047F0000CD0080E4C6209D0000EF86E2D0EF76E2C
:104800004A0EF66EAEEC0DF000D0120001EC21F075
:10481000030E4C6402D0010E6C6F030E4C6202D08A
:10482000020E6C6F020E4C6202D0030E6C6F010E12
:104830004C6202D0040E6C6F000E4C6202D0040E6B
:104840006C6F1200BAC161F0BBC162F0BCC163F011
:10485000BDC164F0BEC165F033EC21F0060E6B6F94
:10486000010E6C6F03EC1DF027EC1EF002E3020E4C
:104870006C6FFBEC1CF027EC1EF002E3030E6C6F78
:10488000F3EC1CF027EC1EF002E3040E6C6FBEDFAD
:10489000D5EC20F026EC20F0C4C14CF0010E4C62A7
:1048A00009D0000EF86E2D0EF76E560EF66EAEECB9
:1048B0000DF024D0020E4C6209D0000EF86E2D0EC1
:1048C000F76E5A0EF66EAEEC0DF018D0030E4C6279
:1048D00009D0000EF86E2D0EF76E5E0EF66EAEEC81
:1048E0000DF00CD0040E4C6209D0000EF86E2D0EA7
:1048F000F76E620EF66EAEEC0DF000D01200AAC19B
:1049000061F0ABC162F0ACC163F0ADC164F0AEC1A7
:1049100065F033EC21F0050E6B6F020E6C6FD5EC79
:1049200020F001EC21F0030E4C6004D0040E6B6FFC
:10493000020E6C6F020E4C6404D0040E6B6F010EFD
:104940006C6F24D0AAC161F0ABC162F0ACC163F05E
:10495000ADC164F0AEC165F033EC21F0040E6B6FB5
:10496000010E6C6FD5EC20F001EC21F0030E4C60D1
:1049700004D0030E6B6F010E6C6F020E4C6406D0F8
:10498000040E6B6F000E6C6FD5EC20F06E8526EC7C
:1049900020F0000EF86E2D0EF76E660EF66EAEEC81
:1049A0000DF01200AFC161F0B0C162F0B1C163F0AF
:1049B000B2C164F0B3C165F033EC21F0040E6B6F4B
:1049C000010E6C6FF3EC1CF027EC1EF003E3030EFA
:1049D0006C6F0FD0FBEC1CF027EC1EF003E3020E13
:1049E0006C6F07D003EC1DF027EC1EF002E3010E04
:1049F0006C6FD5EC20F065D826EC20F0B9C14CF0F6
:104A0000030E4C6209D0000EF86E2D0EF76E360EB6
:104A1000F66EAEEC0DF054D0040E4C6209D0000ED0
:104A2000F86E2D0EF76E3A0EF66EAEEC0DF048D025
:104A3000050E4C6209D0000EF86E2D0EF76E3E0E7C
:104A4000F66EAEEC0DF03CD0060E4C6209D0000EB6
:104A5000F86E2D0EF76E420EF66EAEEC0DF030D005
:104A6000070E4C6209D0000EF86E2D0EF76E460E42
:104A7000F66EAEEC0DF024D0020E4C6209D0000EA2
:104A8000F86E2D0EF76E4E0EF66EAEEC0DF018D0E1
:104A9000010E4C6209D0000EF86E2D0EF76E520E0C
:104AA000F66EAEEC0DF00CD0080E4C6209D0000E84
:104AB000F86E2D0EF76E4A0EF66EAEEC0DF000D0CD
:104AC000120001EC21F0030E4C6404D0050E6B6F54
:104AD000000E6C6F030E4C6202D0010E6C6F020E62
:104AE0004C6202D0020E6C6F010E4C6202D0030EBB
:104AF0006C6F000E4C6202D0030E6C6F1200AFC1DF
:104B000061F0B0C162F0B1C163F0B2C164F0B3C191
:104B100065F033EC21F0030E6B6F010E6C6FF3EC5C
:104B20001CF027EC1EF003E3020E6C6F11D0FBECBF
:104B30001CF027EC1EF003E3010E6C6F09D003ECB0
:104B40001DF027EC1EF004E3000E6C6F040E6B6F7B
:104B5000D5EC20F065D826EC20F0B9C14CF0030E5E
:104B60004C6209D0000EF86E2D0EF76E360EF66E02
:104B7000AEEC0DF054D0040E4C6209D0000EF86E6D
:104B80002D0EF76E3A0EF66EAEEC0DF048D0050E17
:104B90004C6209D0000EF86E2D0EF76E3E0EF66ECA
:104BA000AEEC0DF03CD0060E4C6209D0000EF86E53
:104BB0002D0EF76E420EF66EAEEC0DF030D0070EF5
:104BC0004C6209D0000EF86E2D0EF76E460EF66E92
:104BD000AEEC0DF024D0020E4C6209D0000EF86E3F
:104BE0002D0EF76E4E0EF66EAEEC0DF018D0010ED7
:104BF0004C6209D0000EF86E2D0EF76E520EF66E56
:104C0000AEEC0DF00CD0080E4C6209D0000EF86E20
:104C10002D0EF76E4A0EF66EAEEC0DF000D01200BF
:104C200001EC21F0030E4C6404D0040E6B6F000EF7
:104C30006C6F030E4C6204D0040E6B6F000E6C6F31
:104C4000020E4C6202D0010E6C6F010E4C6202D05B
:104C5000020E6C6F000E4C6202D0020E6C6F1200DE
:104C60004BC161F04CC162F04DC163F04EC164F0C4
:104C70004FC165F055C166F056C167F057C168F085
:104C800058C169F059C16AF08CEC1BF061C04BF15E
:104C900062C04CF163C04DF164C04EF165C04FF18C
:104CA00050C161F051C162F052C163F053C164F070
:104CB00054C165F05AC166F05BC167F05CC168F031
:104CC0005DC169F05EC16AF08CEC1BF061C050F10F
:104CD00062C051F163C052F164C053F165C054F138
:104CE00012004BC161F04CC162F04DC163F04EC186
:104CF00064F04FC165F055C166F056C167F057C109
:104D000068F058C169F059C16AF086EC1BF061C0C7
:104D10004BF162C04CF163C04DF164C04EF165C00F
:104D20004FF150C161F051C162F052C163F053C103
:104D300064F054C165F05AC166F05BC167F05CC1B4
:104D400068F05DC169F05EC16AF086EC1BF061C07D
:104D500050F162C051F163C052F164C053F165C0BB
:104D600054F112004BC161F04CC162F04DC163F0CF
:104D70004EC164F04FC165F055C166F056C167F091
:104D800057C168F058C169F059C16AF0C9EC1AF00E
:104D900061C00EF162C00FF163C010F164C011F187
:104DA00065C012F150C161F051C162F052C163F0AF
:104DB00053C164F054C165F05AC166F05BC167F03D
:104DC0005CC168F05DC169F05EC16AF0C9EC1AF0BF
:104DD00061C013F162C014F163C015F164C016F133
:104DE00065C017F14BC161F04CC162F04DC163F079
:104DF0004EC164F04FC165F05AC166F05BC167F007
:104E00005CC168F05DC169F05EC16AF0C9EC1AF07E
:104E100061C018F162C019F163C01AF164C01BF1DE
:104E200065C01CF150C161F051C162F052C163F024
:104E300053C164F054C165F055C166F056C167F0C6
:104E400057C168F058C169F059C16AF0C9EC1AF04D
:104E500018C166F019C167F01AC168F01BC169F08A
:104E60001CC16AF08CEC1BF061C050F162C051F1C2
:104E700063C052F164C053F165C054F10EC161F0DA
:104E80000FC162F010C163F011C164F012C165F08E
:104E900013C166F014C167F015C168F016C169F05E
:104EA00017C16AF086EC1BF061C04BF162C04CF197
:104EB00063C04DF164C04EF165C04FF112004BC1AB
:104EC00061F04CC162F04DC163F04EC164F04FC15E
:104ED00065F055C166F056C167F057C168F058C11A
:104EE00069F059C16AF0C9EC1AF061C00EF162C0F4
:104EF0000FF163C010F164C011F165C012F150C12F
:104F000061F051C162F052C163F053C164F054C109
:104F100065F05AC166F05BC167F05CC168F05DC1C5
:104F200069F05EC16AF0C9EC1AF00EC166F00FC1FB
:104F300067F010C168F011C169F012C16AF08CEC21
:104F40001BF061C00EF162C00FF163C010F164C0CC
:104F500011F165C012F155C161F056C162F057C13F
:104F600063F058C164F059C165F055C166F056C18F
:104F700067F057C168F058C169F059C16AF0C9ECCF
:104F80001AF061C013F162C014F163C015F164C07E
:104F900016F165C017F15AC161F05BC162F05CC1E6
:104FA00063F05DC164F05EC165F05AC166F05BC13B
:104FB00067F05CC168F05DC169F05EC16AF0C9EC80
:104FC0001AF013C166F014C167F015C168F016C17C
:104FD00069F017C16AF08CEC1BF061C013F162C07C
:104FE00014F163C015F164C016F165C017F1FBEC54
:104FF00016F00EC161F00FC162F010C163F011C173
:1050000064F012C165F049EC1BF061C00EF162C0A2
:105010000FF163C010F164C011F165C012F14BC112
:1050200061F04CC162F04DC163F04EC164F04FC1FC
:1050300065F05AC166F05BC167F05CC168F05DC1A4
:1050400069F05EC16AF0C9EC1AF061C018F162C083
:1050500019F163C01AF164C01BF165C01CF150C1A5
:1050600061F051C162F052C163F053C164F054C1A8
:1050700065F055C166F056C167F057C168F058C178
:1050800069F059C16AF0C9EC1AF018C166F019C18B
:1050900067F01AC168F01BC169F01CC16AF086ECA8
:1050A0001BF013C166F014C167F015C168F016C19A
:1050B00069F017C16AF049EC1BF061C050F162C0A1
:1050C00051F163C052F164C053F165C054F10EC197
:1050D0004BF10FC14CF110C14DF111C14EF112C194
:1050E0004FF112004BC15FF14CC160F14DC161F154
:1050F0004EC162F14FC163F150C164F151C165F11C
:1051000052C166F153C167F154C168F112005FC129
:105110004BF160C14CF161C14DF162C14EF163C10F
:105120004FF164C150F165C151F166C152F167C1DF
:1051300053F168C154F1120055C169F156C16AF1C9
:1051400057C16BF158C16CF159C16DF15AC16EF183
:105150005BC16FF15CC170F15DC171F15EC172F153
:10516000120069C155F16AC156F16BC157F16CC1AA
:1051700058F16DC159F16EC15AF16FC15BF170C147
:105180005CF171C15DF172C15EF1120072EC28F048
:105190009CEC28F030EC26F04BC173F14CC174F15B
:1051A0004DC175F14EC176F14FC177F150C178F123
:1051B00051C179F152C17AF153C17BF154C17CF1F3
:1051C00087EC28F0B1EC28F0B2EC26F073C155F171
:1051D00074C156F175C157F176C158F177C159F1D3
:1051E00078C15AF179C15BF17AC15CF17BC15DF1A3
:1051F0007CC15EF15FEC27F012008EEC0DF074ECD8
:1052000029F002EC0CF012008EEC0DF04BC161F0B5
:105210004CC162F04DC163F04EC164F04FC165F006
:105220006551A0EC0DF06451A0EC0DF06351A0ECC1
:105230000DF06251A0EC0DF06151A0EC0DF098EC76
:105240000DF050C161F051C162F052C163F053C121
:1052500064F054C165F06551A0EC0DF06451A0EC10
:105260000DF06351A0EC0DF06251A0EC0DF0615116
:10527000A0EC0DF0400E96EC0DF055C161F056C15A
:1052800062F057C163F058C164F059C165F06551CF
:10529000A0EC0DF06451A0EC0DF06351A0EC0DF00A
:1052A0006251A0EC0DF06151A0EC0DF098EC0DF006
:1052B0005AC161F05BC162F05CC163F05DC164F032
:1052C0005EC165F06551A0EC0DF06451A0EC0DF0ED
:1052D0006351A0EC0DF06251A0EC0DF06151A0EC17
:1052E0000DF002EC0CF01200000E4BC161F04CC14D
:1052F00062F04DC163F04EC164F04FC165F00FD84C
:10530000400E50C161F051C162F052C163F053C10F
:1053100064F054C165F003D86A0E09EF0DF096EC05
:105320000DF033EC21F00D0E6B6F070E6C6F6E8578
:10533000D5EC20F026EF20F0400E4BC161F04CC1BF
:1053400062F04DC163F04EC164F04FC165F0E7DF1C
:10535000140E50C161F051C162F052C163F053C1EB
:1053600064F054C165F0DBDF6A0E09EF0DF0140E36
:105370004BC161F04CC162F04DC163F04EC164F0AD
:105380004FC165F0CCDF540E50C161F051C162F0E5
:1053900052C163F053C164F054C165F0C0DF6A0EBE
:0453A00009EF0DF014
:020000040030CA
:0300010022193C85
:020005003D803C
:0200000400F00A
:020000000401F9
:00000001FF
